:100000000C942A001895000018950000189500001F
:10001000189500001895000018950000189500002C
:10002000189500000C9434011895000018950000F4
:10003000189500001895000018950000189500000C
:1000400018950000189500001895000018950000FC
:10005000189500008FE58DBFC0E4E6E24E2E88E0E3
:100060008EBFD8E0F8E05F2EEEEFF7E0A0E6B0E05C
:1000700088278D933197E9F784B7082E877F84BF4F
:100080008FE181BD87E081BD662487E886B980E085
:1000900087B98FEF84BB80E08FBD84E08EBD89B7C8
:1000A000846089BF7894AA9A379A40916100009140
:1000B0006000041711F40C94300107B1007E046055
:1000C00007B90E947F01A2E6B0E08D939C9307B12F
:1000D000007E056007B90E947F01A4E6B0E08D9321
:1000E0009C9307B1007E066007B90E947F01A6E6D7
:1000F000B0E08D939C9307B1007E076007B90E9422
:100100007F01A8E6B0E08D939C93A2E6B0E00D914C
:100110001C91A4E6B0E04D915C91040F151FAAE676
:10012000B0E00D931C93A6E6B0E00D911C91A8E6FB
:10013000B0E04D915C91040F151FACE6B0E00D935B
:100140001C93AAE6B0E00D911C91ACE6B0E04D9195
:100150005C91040F151FAEE6B0E00D931C93AEE664
:10016000B0E00D911C91043F51E0150718F011F01B
:100170000C94BC000C941401AA980091600001300A
:1001800018F011F00C940E01A4E6B0E04D915C91D2
:10019000A2E6B0E00D911C910417150718F011F0BC
:1001A0000C94D4000C94D600AE9AAF98A2E6B0E0BE
:1001B0004D915C91A4E6B0E00D911C9104171507D8
:1001C00018F011F00C94E6000C94E800AF9AAE9889
:1001D000A8E6B0E04D915C91A6E6B0E00D911C91CF
:1001E0000417150718F011F00C94F8000C94FA009D
:1001F000AC9AAD98A6E6B0E04D915C91A8E6B0E06F
:100200000D911C910417150718F011F00C940A01B8
:100210000C940C01AD9AAC980C941201AC9AAD9A66
:10022000AE9AAF9A0C942301AEE6B0E00D911C910A
:10023000043B50E0150710F00C942301AA9AAE9AE3
:10024000AF98AC9AAD9800916000053011F00C9415
:100250002C0180E0809360008091600080936100B9
:100260000C945500F894FFCF0F921F922F923F925B
:100270004F925F927F92AF92BF920F931F932F93F3
:100280003F934F935F936F937F938F939F93AF931E
:10029000BF93CF93DF93EF93FF938FB78F938CED43
:1002A0009BE090934D0080934C00A0E6B0E08C91D1
:1002B0008F5F8C938F918FBFFF91EF91DF91CF91E3
:1002C000BF91AF919F918F917F916F915F914F916E
:1002D0003F912F911F910F91BF90AF907F905F90B2
:1002E0004F903F902F901F900F9018953197F1F7F6
:1002F0000895689462F80895E89462F80895369A2B
:100300003699FECF369A3699FECF84B195B10895CD
:00000001FF
